:020000040000FA
:100000000C9490000C94B8000C94B8000C94B800B8
:100010000C94B8000C94B8000C94B8000C94B80080
:100020000C94B8000C94B8000C94B8000C94B80070
:100030000C94B8000C94B8000C94B8000C94B80060
:100040000C94D3090C94B8000C94A1090C947B096E
:100050000C94B8000C94B8000C94B8000C94B80040
:100060000C94B8000C94B80008000000BE9224491B
:10007000123EABAAAA2ABECDCCCC4C3E00000080DA
:10008000BEABAAAAAA3E00000000BF000000803F4D
:100090000000000000084178D3BB4387D1133D190D
:1000A0000E3CC3BD4282AD2B3E68EC8276BED98F3A
:1000B000E1A93E4C80EFFFBE01C4FF7F3F0000007E
:1000C000000000000000240027002A0000000000BB
:1000D000250028002B000000000023002600290036
:1000E00004040404040404040202020202020303DE
:1000F00003030303010204081020408001020408E6
:100100001020010204081020000000080002010075
:100110000003040700000000000000001D0AF90CA5
:1001200011241FBECFEFD8E0DEBFCDBF24E0A2E296
:10013000B4E001C01D92A03FB207E1F714E0A0E0D7
:10014000B1E0EAE4F4E202C005900D92A232B107F8
:10015000D9F710E0CFE8D0E004C02197FE010E945B
:100160001710CE38D107C9F70E94580A0C941812FC
:100170000C940000AF92BF92CF92DF92EF92FF9269
:100180000F931F93CF93DF936C017B018B01040FBF
:10019000151FEB015E01AE18BF08C017D10759F05B
:1001A0006991D601ED91FC910190F081E02DC6019D
:1001B0000995892B79F7C501DF91CF911F910F9197
:1001C000FF90EF90DF90CF90BF90AF900895FC012B
:1001D000538D448D252F30E0842F90E0821B930BAC
:1001E000541710F0CF96089501970895FC01918D52
:1001F000828D981761F0A28DAE0FBF2FB11D5D9655
:100200008C91928D9F5F9F73928F90E008958FEFF6
:100210009FEF0895FC01918D828D981731F0828DAA
:10022000E80FF11D858D90E008958FEF9FEF089501
:10023000FC01918D228D892F90E0805C9F4F821B65
:1002400091098F739927089589E494E00E94180119
:1002500021E0892B09F420E0822F089580E090E0CE
:10026000892B29F00E94240181110C94000008952B
:10027000FC01A48DA80FB92FB11DA35ABF4F2C911B
:10028000848D90E001968F739927848FA689B78912
:100290002C93A089B1898C91837080648C93938D09
:1002A000848D981306C00288F389E02D80818F7DAC
:1002B00080830895EF92FF920F931F93CF93DF9364
:1002C000EC0181E0888F9B8D8C8D98131AC0E88992
:1002D000F989808185FF15C09FB7F894EE89FF8961
:1002E0006083E889F98980818370806480839FBFFF
:1002F00081E090E0DF91CF911F910F91FF90EF90FF
:100300000895F62E0B8D10E00F5F1F4F0F7311270E
:10031000E02E8C8D8E110CC00FB607FCFACFE88949
:10032000F989808185FFF5CFCE010E943801F1CF98
:10033000EB8DEC0FFD2FF11DE35AFF4FF0829FB7BD
:10034000F8940B8FEA89FB8980818062CFCFCF93AD
:10035000DF93EC01888D8823B9F0AA89BB89E889ED
:10036000F9898C9185FD03C0808186FD0DC00FB693
:1003700007FCF7CF8C9185FFF2CF808185FFEDCF11
:10038000CE010E943801E9CFDF91CF9108958330EB
:1003900081F028F4813099F08230A9F008958730F7
:1003A000A9F08830C9F08430B1F4809180008F7D4D
:1003B00003C0809180008F7780938000089584B57A
:1003C0008F7784BD089584B58F7DFBCF8091B00079
:1003D0008F778093B00008958091B0008F7DF9CF22
:1003E000CF93DF93282F30E0F901E85FFE4F84912F
:1003F000F901EC50FF4FD491F901E052FF4FC49145
:10040000CC23A1F081110E94C701EC2FF0E0EE0F88
:10041000FF1FEA52FF4FA591B491EC91ED2381E0CB
:1004200090E009F480E0DF91CF91089580E090E0C2
:10043000FACF1F93CF93DF93282F30E0F901E85FC5
:10044000FE4F8491F901EC50FF4FD491F901E05235
:10045000FF4FC491CC23A9F0162F81110E94C70130
:10046000EC2FF0E0EE0FFF1FE453FF4FA591B49186
:100470008FB7F894EC91111108C0D095DE23DC936E
:100480008FBFDF91CF911F910895DE2BF8CFCF93CF
:10049000DF9390E0FC01EC50FF4F249180529F4F7E
:1004A000FC0184918823D1F090E0880F991FFC0112
:1004B000EE53FF4FA591B491FC01E453FF4FC5915A
:1004C000D49161110EC09FB7F8948C91E22FE09502
:1004D0008E238C932881E223E8839FBFDF91CF9105
:1004E00008958FB7F894EC91E22BEC938FBFF6CF81
:1004F0003FB7F89480913B0490913C04A0913D0457
:10050000B0913E0426B5A89B05C02F3F19F0019677
:10051000A11DB11D3FBFBA2FA92F982F8827BC015D
:10052000CD01620F711D811D911D42E0660F771F85
:10053000881F991F4A95D1F708958F929F92AF9285
:10054000BF92CF92DF92EF92FF924B015C010E942B
:1005500078026B017C010E9478026C197D098E097A
:100560009F09683E734081059105A8F321E0821A36
:100570009108A108B10888EEC80E83E0D81EE11CDE
:10058000F11C81149104A104B10429F7FF90EF90AC
:10059000DF90CF90BF90AF909F908F9008952FB72E
:1005A000F8946091370470913804809139049091E7
:1005B0003A042FBF0895FC0101900020E9F731971C
:1005C000AF01481B590BBC0189E494E00C94BA00BC
:1005D000009711F00C94DB0290E080E008958F9278
:1005E0009F92AF92BF920F931F93CF93DF93CDB79C
:1005F000DEB7A1970FB6F894DEBF0FBECDBF19A22C
:10060000423008F44AE08E010F5D1F4F842E912C7A
:10061000B12CA12CA50194010E94F50FE62FB90180
:10062000CA01EA30D4F4E05DD801EE938D01232BAA
:10063000242B252B79F7CD010E94E802A1960FB655
:10064000F894DEBF0FBECDBFDF91CF911F910F9108
:10065000BF90AF909F908F900895E95CE5CF60E0E8
:100660008CE00E94190264E670E080E090E00E9455
:100670009D028CE191E00E94E80261E088E00E9426
:10068000190280910201909103018230910564F07A
:100690000197909303018093020168EE73E080E07C
:1006A00090E00E949D02EDCF60E088E00E94190278
:1006B00064E670E080E090E00E949D028EE291E0AE
:1006C0000E94E80261E08CE00C941902CF92DF9264
:1006D000EF92FF9260E08CE00E94190264E670E005
:1006E00080E090E00E949D0282E491E00E94E80296
:1006F00061E08AE00E9419026CED75E080E090E014
:100700000E949D0260E08AE00E94190261E08BE095
:100710000E9419020E94CF026B017C01C092430427
:10072000D0924404E0924504F09246046AE070E0FE
:1007300080E090E00E949D0284E00E94F001019719
:10074000E1F46CED75E080E090E00E949D0260E0D5
:100750008BE00E94190264E670E080E090E00E9465
:100760009D0281E591E00E94E80261E08CE0FF904B
:10077000EF90DF90CF900C9419020E94CF026C1979
:100780007D098E099F0969397A438105910570F2C7
:1007900064E670E080E090E00E949D028CE591E0CC
:1007A0000E94E80260E08BE00E94190281E090E084
:1007B0009093480480934704D8CFCF92DF92EF9272
:1007C000FF9260E08CE00E94190264E670E080E035
:1007D00090E00E949D028EE791E00E94E80261E0B5
:1007E0008BE00E94190268EE73E080E090E00E94C6
:1007F0009D0260E08BE00E94190261E08AE00E94A5
:1008000019020E94CF026B017C01C0924304D09276
:100810004404E0924504F09246046AE070E080E00F
:1008200090E00E949D0283E00E94F0010197E1F4B4
:1008300064E873E080E090E00E949D0260E08AE05E
:100840000E94190264E670E080E090E00E949D0240
:1008500083E591E00E94E80261E08CE0FF90EF9078
:10086000DF90CF900C9419020E94CF026C197D0981
:100870008E099F0969397A438105910570F264E612
:1008800070E080E090E00E949D028BE891E00E9481
:10089000E80260E08AE00E94190281E090E0909313
:1008A000480480934704D8CF60E08CE00E9419028E
:1008B00064E670E080E090E00E949D028BEA91E0A7
:1008C0000E94E80261E087E00E94190268EE73E08E
:1008D00080E090E00E949D0260E087E00E941902A3
:1008E00064E670E080E090E00E949D0288EB91E079
:1008F0000E94E80261E08CE00C941902CF92DF9232
:10090000EF92FF9260E08CE00E94190264E670E0D2
:1009100080E090E00E949D0281EC91E00E94E8025C
:1009200061E089E00E9419020E94CF026B017C0104
:10093000C0924304D0924404E0924504F0924604ED
:100940006AE070E080E090E00E949D0282E00E94F8
:10095000F0010197B1F460E089E00E94190264E6B9
:1009600070E080E090E00E949D028EEC91E00E9499
:10097000E80261E08CE0FF90EF90DF90CF900C9464
:1009800019020E94CF026C197D098E099F096939ED
:100990007A4381059105A0F28DED91E00E94E80275
:1009A00060E089E00E94190264E670E080E090E077
:1009B0000E949D028FEF91E00E94E80281E090E0AA
:1009C00090933504809334049093330480933204DD
:1009D000D0CFFC0180819181009711F00C94B91067
:1009E0000895FC0124813581232B39F421E0FB019A
:1009F0008081882349F020E007C0808191810E9496
:100A0000081221E0892BB9F7822F08950F931F93C5
:100A1000CF93DF93EC0188819981009759F02A8167
:100A20003B812617370730F081E0DF91CF911F918E
:100A30000F9108958B016F5F7F4F0E9442110097C5
:100A400059F0998388831B830A832C813D81232B52
:100A500059F7FC011082E8CF80E0E7CFEF92FF92D8
:100A60000F931F93CF93DF93EC017B018A01BA01AF
:100A70000E94060528813981811114C02115310594
:100A800019F0C9010E94B910198218821D821C82B6
:100A90001B821A82CE01DF91CF911F910F91FF909F
:100AA000EF9008951D830C83B701C9010E941112B4
:100AB000F1CFFB0101900020E9F73197AF01461B10
:100AC000570B0C942E05FF920F931F93CF93DF9338
:100AD000EC01198218821B821A821D821C8250E04E
:100AE00040E06BEB73E00E942E050091EA04109148
:100AF000EB0401151105F9F00430110510F004E0C4
:100B000010E0E091E604F091E704E00FF11FF080BF
:100B100010826091E6047091E7046115710591F00F
:100B2000CE010E9459058091E6049091E704080FD8
:100B3000191FF801F082CE01DF91CF911F910F9123
:100B4000FF90089588819981009711F00E94B91053
:100B5000198218821D821C821B821A82E4CF0F9395
:100B60001F93CF93DF9300D0CDB7DEB789E494E035
:100B70000E941801892BA1F16AE070E080E090E00A
:100B80000E949D0289E494E00E941801181619063B
:100B90006CF789E494E00E94F60089831A82009140
:100BA000EA041091EB040F5F1F4FB80186EE94E04A
:100BB0000E9406058823D1F22091E6043091E704D3
:100BC0008091EA049091EB04BE016F5F7F4F820F2A
:100BD000931F0E9411121093EB040093EA04C6CFF6
:100BE0000F900F90DF91CF911F910F9108958F92E9
:100BF0009F92AF92BF92CF92DF92EF92FF921F939C
:100C0000CF93DF9360E08CE00E94190261E08DE0F9
:100C10000E9419020E94CF0260934304709344041F
:100C2000809345049093460460932E0470932F04A0
:100C3000809330049093310464E670E080E090E0AB
:100C40000E949D028FE092E00E94E80264E670E05C
:100C500080E090E00E949D02C0900001D0900101D0
:100C60000D2C000CEE08FF084AE0C701B601F7FEA4
:100C70000DC06DE289E494E00E945A01662777274F
:100C8000CB016C197D098E099F094AE00E94EF0291
:100C900064E670E080E090E00E949D0210922A04D9
:100CA00010922B0410922C0410922D0480E090E0FE
:100CB000A0E2B1EC8093260490932704A09328042B
:100CC000B093290480E090E0A8ECB2EC8093220479
:100CD00090932304A0932404B093250417E4109365
:100CE0007C0080917A00806480937A0080917A0001
:100CF00086FDFCCF8091780060917900762F682F77
:100D0000072E000C880B990B0E94040D9B01AC016F
:100D100060E070EC8FE794E40E94C50E20E030E0C4
:100D200040E85FE30E94580E20E030E44CE156E4D6
:100D30000E94630D0E94730F6B017C0125E93FEB5C
:100D400046E554E30E94630DA70196010E94630DDE
:100D5000A70196010E94630D4B015C012FE83CEF57
:100D600041E459E3C701B6010E94630D29E832ED61
:100D70004EE55AE30E94590E9B01AC01C501B40136
:100D80000E94590E9B01AC0160E070E080E89FE397
:100D90000E94C50E23E333E948E853E40E94580E4D
:100DA0006B017C01C0922A04D0922B04E0922C04A7
:100DB000F0922D040E94CF0280904304909044044E
:100DC000A0904504B0904604681979098A099B09E6
:100DD000683E73408105910541F4C0922204D0928F
:100DE0002304E0922404F0922504C0910001D091E4
:100DF0000101BE010D2E000C880B990B0E94040D01
:100E00009B01AC01C701B6010E94660F18160CF0D9
:100E1000CDC064E670E080E090E00E949D028BE12E
:100E200092E00E94E80264E670E080E090E00E94B8
:100E30009D02C0902A04D0902B04E0902C04F090E6
:100E40002D04A7019601C701B6010E94BB0F88239C
:100E5000D9F081E392E00E94DB0260E086E00E942C
:100E6000190260E08DE00E94190261E08CE0DF91E0
:100E7000CF911F91FF90EF90DF90CF90BF90AF90F8
:100E80009F908F900C94190246015701E894B7F88F
:100E90002FEF3FEF4FE75FE7C501B4010E94BB0FA3
:100EA00081110DC02FEF3FEF4FE75FE7C501B401A0
:100EB0000E94FD0C18161CF485E392E0CCCF2FEFB6
:100EC0003FEF4FE75FE4C701B6010E94660F1816B7
:100ED0001CF489E392E0BFCF2FEF3FEF4FE75FECC9
:100EE000C701B6010E94FD0C87FDF3CF20E030E082
:100EF000A901C701B6010E94FD0C87FF09C06DE280
:100F000089E494E00E945A01F7FAF094F7F8F0941B
:100F10002AE037ED43EA5BE3C701B6010E94590EB0
:100F20004B015C010E94370F6B017C010E94020D96
:100F30009B01AC01C501B4010E94580E4B015C013C
:100F40004AE0C701B6010E94EF026EE289E494E034
:100F50000E945A0120E030E040E251E4C501B401B2
:100F60000E94630D4B015C010E94370F6B01F12C55
:100F7000E12C4AE0C701B6010E94EF02C701B601A9
:100F80000E94020D9B01AC01C501B4010E94580EE4
:100F900020E030E040E251E40E94630D0E94370FF0
:100FA00090E080E04AE00E94EF0257CF20E030E07E
:100FB00048EC52ECC701B6010E94FD0C87FF11C03E
:100FC00064E670E080E090E00E949D028DE392E094
:100FD0000E94E80281E090E09093480480934704E7
:100FE0003CCF0E94CF02681979098A099B096132B6
:100FF0007E4481059105E8F020912204309123047C
:101000004091240450912504C701B6010E94580E56
:1010100020E030E040E85FE30E94FD0C87FF09C05C
:1010200064E670E080E090E00E949D0282E692E03B
:10103000CFCF0E94CF02681979098A099B096136CE
:101040007A4E8105910558F064E670E080E090E00A
:101050000E949D028EE892E00E94E802FECE0E946D
:10106000CF02AB01BC0180912E0490912F04A0917E
:101070003004B091310488519C4FAF4FBF4F84175B
:101080009507A607B70738F5BE0164517109072E09
:10109000000C880B990B0E94040D9B01AC01C70149
:1010A000B6010E94FD0C87FF1DC061E086E00E9432
:1010B0001902C0922604D0922704E0922804F092EC
:1010C00029040E94CF0260932E0470932F04809312
:1010D0003004909331046AE070E080E090E00E9478
:1010E0009D02FDCD209126043091270440912804D3
:1010F00050912904C701B6010E94580E20E030E04B
:1011000040E05FE30E94FD0C87FDCFCF60E0CECFD3
:10111000CF93DF9300D000D000D0CDB7DEB785E508
:1011200090E090930101809300010E94F705809167
:10113000470490914804019709F4CFC0809141047D
:1011400090914204892B41F480913F049091400496
:10115000892B11F40E947E0480913404909135040F
:10116000019709F043C064E670E080E090E00E94DF
:101170009D0280EB92E00E94E80289E494E00E94E4
:10118000180118161906CCF76BEB73E086EE94E0A5
:101190000E9459050E94AF05CE0101960E94630589
:1011A00065ED72E0CE0101960E94F104882309F4F6
:1011B0009DC08AED92E00E94E802109235041092E0
:1011C00034040E947E04809134049091350481306F
:1011D000910541F4909348048093470484EE92E093
:1011E0000E94E802CE0101960E94E9048091470422
:1011F00090914804019709F470C068EE73E080E0B4
:1012000090E00E949D020E946603809147049091A5
:101210004804019709F461C00E94540468EE73E029
:1012200080E090E00E949D020E94DD0380914704CF
:1012300090914804019709F450C08FE590E0909395
:101240000101809300010E94F7058091470490916D
:101250004804019709F441C08091410490914204EF
:10126000892B61F464E670E080E090E00E949D02CA
:101270000E942F0360E086E00E94190268EB7BE089
:1012800080E090E00E949D020E94660380914704E6
:1012900090914804019709F164E670E080E090E0E5
:1012A0000E949D0288E193E00E94E80268EE73E0EC
:1012B00080E090E00E949D0210924204109241044E
:1012C0001092400410923F048091320490913304B4
:1012D000019719F4F0E0E0E0099526960FB6F8942E
:1012E000DEBF0FBECDBFDF91CF910895CE01019635
:1012F0000E94E90442CF1F920F920FB60F92112461
:101300002F933F934F935F936F937F938F939F930D
:10131000AF93BF93EF93FF9389E494E00E94380169
:10132000FF91EF91BF91AF919F918F917F916F91BD
:101330005F914F913F912F910F900FBE0F901F9093
:1013400018951F920F920FB60F9211242F938F931F
:101350009F93EF93FF93E0915904F0915A04808199
:10136000E0915F04F091600482FD1BC09081809148
:1013700062048F5F8F7320916304821741F0E091C4
:101380006204F0E0E75BFB4F958F80936204FF916E
:10139000EF919F918F912F910F900FBE0F901F9003
:1013A00018958081F4CF1F920F920FB60F921124DF
:1013B0002F933F938F939F93AF93BF938091370465
:1013C00090913804A0913904B0913A0430913604D8
:1013D00023E0230F2D3758F50196A11DB11D209351
:1013E00036048093370490933804A0933904B09363
:1013F0003A0480913B0490913C04A0913D04B0914B
:101400003E040196A11DB11D80933B0490933C04C2
:10141000A0933D04B0933E04BF91AF919F918F91F3
:101420003F912F910F900FBE0F901F90189526E8B7
:10143000230F0296A11DB11DD2CFE9E4F4E013827F
:10144000128288EE93E0A0E0B0E084839583A683C7
:10145000B7838EE091E09183808385EC90E095875F
:10146000848784EC90E09787868780EC90E0918B6E
:10147000808B81EC90E0938B828B82EC90E0958B5B
:10148000848B86EC90E0978B868B118E128E138E58
:10149000148EE6EEF4E0118210821382128215821D
:1014A000148250E040E06BEB73E0CF010C942E050A
:1014B000CF93DF9300D000D000D0CDB7DEB77894C3
:1014C00084B5826084BD84B5816084BD85B5826049
:1014D00085BD85B5816085BD80916E0081608093FA
:1014E0006E00109281008091810082608093810063
:1014F0008091810081608093810080918000816073
:10150000809380008091B10084608093B1008091CD
:10151000B00081608093B00080917A0084608093F5
:101520007A0080917A00826080937A0080917A00BC
:10153000816080937A0080917A00806880937A003D
:101540001092C10061E086E00E94470261E088E0FD
:101550000E94470261E089E00E94470261E087E063
:101560000E94470261E08AE00E94470261E08BE04E
:101570000E94470261E08DE00E94470261E08CE03A
:101580000E94470260E082E00E94470260E085E03E
:101590000E94470260E085E10E94470260E084E02B
:1015A0000E94470260E083E00E94470260E089E019
:1015B0000E94190260E088E00E94190260E086E063
:1015C0000E94190260E087E00E94190260E08AE050
:1015D0000E94190260E08BE00E94190260E08DE039
:1015E0000E94190260E08CE00E941902E091590407
:1015F000F0915A0482E08083E0915504F091560402
:101600001082E0915704F09158048FEC808310927F
:101610006104E0915D04F0915E0486E08083E091D6
:101620005B04F0915C04808180618083E0915B04C5
:10163000F0915C04808188608083E0915B04F0918C
:101640005C04808180688083E0915B04F0915C049D
:1016500080818F7D808364E670E080E090E00E946E
:101660009D0283E293E00E94E80201E010E040E581
:10167000242E312C5FE0E52EF12C64E6462E512C11
:101680008CE3C82ED12C99E1A92EB12C24E1822E15
:10169000912C30E0632E30E0732E61E08CE00E94EC
:1016A00019028091470490914804019709F04CC0B9
:1016B0000E94CF02609343047093440480934504D6
:1016C0009093460464E670E080E090E00E949D0202
:1016D00087E393E00E94E80264E670E080E090E037
:1016E0000E949D028CE493E00E94E80260E08CE09E
:1016F0000E94190261E08DE00E94190268EE73E019
:1017000080E090E00E949D0260E08DE00E9419025E
:1017100068EE73E080E090E00E949D020E94CF029C
:101720002091430430914404409145045091460473
:10173000621B730B840B950B603375478105910514
:10174000C9F6F0E0E0E0099589E494E00E94180110
:10175000181619060CF01AC16BEB73E086EE94E0D4
:101760000E9459050E94AF05CE0101960E946305B3
:1017700067E673E0CE0101960E94F104882371F0C0
:1017800064E670E080E090E00E949D028CE693E0C9
:101790000E94E802F0920301E092020167E773E021
:1017A000CE0101960E94F104882371F064E670E096
:1017B00080E090E00E949D028CE793E00E94E802A6
:1017C000909203018092020166E873E0CE010196D7
:1017D0000E94F104882371F064E670E080E090E0FC
:1017E0000E949D028BE893E00E94E802B092030100
:1017F000A092020162E973E0CE0101960E94F10419
:10180000882371F064E670E080E090E00E949D0221
:1018100087E993E00E94E802D0920301C09202019E
:1018200062EA73E0CE0101960E94F104882361F020
:1018300064E670E080E090E00E949D0287EA93E019
:101840000E94E8020E9488086CEB73E0CE010196CA
:101850000E94F104882381F064E670E080E090E06B
:101860000E949D0281EC93E00E94E80210934204E2
:10187000009341040E94880869EC73E0CE01019650
:101880000E94F1048823B1F064E670E080E090E00B
:101890000E949D028EEC93E00E94E8028CE090E0B2
:1018A00090930301809302011093400400933F043E
:1018B0000E94880864ED73E0CE0101960E94F10455
:1018C00081110E947E0469ED73E0CE0101960E94B1
:1018D000F104882331F0F0920301E09202010E94AA
:1018E0002F036EED73E0CE0101960E94F104811189
:1018F0000E94DD0363EE73E0CE0101960E94F104C5
:1019000081110E94660368EE73E0CE0101960E9489
:10191000F104882331F030920101209200010E94ED
:10192000F7056DEE73E0CE0101960E94F10481117E
:101930000E94540462EF73E0CE0101960E94F1040C
:10194000882301F164E670E080E090E00E949D024F
:1019500087EF93E00E94E802109342040093410451
:101960000E9488081093400400933F040E94880856
:1019700064E670E080E090E00E949D0280E094E0E8
:101980000E94E802CE0101960E94E90485E00E94CF
:10199000F0010197E1F4509201014092000182E1CF
:1019A00094E00E94E80264EF71E080E090E00E9421
:1019B0009D020E94F70560E27EE480E090E00E94D4
:1019C0009D0280914704909148040197F9F66AE0DE
:1019D00070E080E090E00E949D026114710409F4BF
:1019E0005CCE0E942401882309F44ACE0E940000A4
:1019F00047CE86EE94E00C94E9040E943F0D08F473
:101A000081E00895E89409C097FB3EF49095809595
:101A1000709561957F4F8F4F9F4F9923A9F0F92FB4
:101A200096E9BB279395F695879577956795B79532
:101A3000F111F8CFFAF4BB0F11F460FF1BC06F5F18
:101A40007F4F8F4F9F4F16C0882311F096E911C02A
:101A5000772321F09EE8872F762F05C0662371F04B
:101A600096E8862F70E060E02AF09A95660F771F5F
:101A7000881FDAF7880F9695879597F90895990F3B
:101A80000008550FAA0BE0E8FEEF16161706E80748
:101A9000F907C0F012161306E407F50798F0621B69
:101AA000730B840B950B39F40A2661F0232B242B3E
:101AB000252B21F408950A2609F4A140A6958FEF5D
:101AC000811D811D08950E94760D0C94E70D0E94E2
:101AD000D90D38F00E94E00D20F0952311F00C9400
:101AE000D00D0C94D60D11240C941B0E0E94F80DF1
:101AF00070F3959FC1F3950F50E0551F629FF00161
:101B0000729FBB27F00DB11D639FAA27F00DB11D79
:101B1000AA1F649F6627B00DA11D661F829F222702
:101B2000B00DA11D621F739FB00DA11D621F839F89
:101B3000A00D611D221F749F3327A00D611D231F5F
:101B4000849F600D211D822F762F6A2F11249F57AD
:101B500050409AF0F1F088234AF0EE0FFF1FBB1FB0
:101B6000661F771F881F91505040A9F79E3F51056F
:101B700080F00C94D00D0C941B0E5F3FE4F3983E64
:101B8000D4F3869577956795B795F795E7959F5F19
:101B9000C1F7FE2B880F911D9695879597F90895AB
:101BA00097F99F6780E870E060E008959FEF80EC10
:101BB000089500240A9416161706180609060895B3
:101BC00000240A9412161306140605060895092E19
:101BD0000394000C11F4882352F0BB0F40F4BF2B88
:101BE00011F460FF04C06F5F7F4F8F4F9F4F0895C8
:101BF00057FD9058440F551F59F05F3F71F04795BE
:101C0000880F97FB991F61F09F3F79F087950895A2
:101C1000121613061406551FF2CF4695F1DF08C0C1
:101C2000161617061806991FF1CF869571056105DE
:101C300008940895E894BB2766277727CB0197F986
:101C400008952F923F924F925F926F927F928F9260
:101C50009F92AF92BF92CF92DF92EF92FF920F933B
:101C60001F93CF93DF93CDB7DEB7CA1BDB0B0FB645
:101C7000F894DEBF0FBECDBF09942A883988488802
:101C80005F846E847D848C849B84AA84B984C88498
:101C9000DF80EE80FD800C811B81AA81B981CE0F8F
:101CA000D11D0FB6F894DEBF0FBECDBFED01089574
:101CB0005058BB27AA270E94700E0C94E70D0E9473
:101CC000D90D38F00E94E00D20F039F49F3F19F44F
:101CD00026F40C94D60D0EF4E095E7FB0C94D00D91
:101CE000E92F0E94F80D58F3BA17620773078407AB
:101CF000950720F079F4A6F50C941A0E0EF4E095F1
:101D00000B2EBA2FA02D0B01B90190010C01CA01B5
:101D1000A0011124FF27591B99F0593F50F4503E60
:101D200068F11A16F040A22F232F342F4427585F52
:101D3000F3CF469537952795A795F0405395C9F76A
:101D40007EF41F16BA0B620B730B840BBAF0915022
:101D5000A1F0FF0FBB1F661F771F881FC2F70EC0C1
:101D6000BA0F621F731F841F48F487957795679594
:101D7000B795F7959E3F08F0B0CF9395880F08F080
:101D80009927EE0F9795879508950E94D90E0C9488
:101D9000E70D0E94E00D58F00E94D90D40F029F4A3
:101DA0005F3F29F00C94D00D51110C941B0E0C9434
:101DB000D60D0E94F80D68F39923B1F3552391F3E2
:101DC000951B550BBB27AA2762177307840738F0AA
:101DD0009F5F5F4F220F331F441FAA1FA9F335D007
:101DE0000E2E3AF0E0E832D091505040E695001CBB
:101DF000CAF72BD0FE2F29D0660F771F881FBB1F75
:101E0000261737074807AB07B0E809F0BB0B802D52
:101E1000BF01FF2793585F4F3AF09E3F510578F07E
:101E20000C94D00D0C941B0E5F3FE4F3983ED4F35A
:101E3000869577956795B795F7959F5FC9F7880F52
:101E4000911D9695879597F90895E1E0660F771FA4
:101E5000881FBB1F621773078407BA0720F0621B35
:101E6000730B840BBA0BEE1F88F7E09508950E9460
:101E7000000E88F09F5798F0B92F9927B751B0F00E
:101E8000E1F0660F771F881F991F1AF0BA95C9F7FE
:101E900014C0B13091F00E941A0EB1E008950C9474
:101EA0001A0E672F782F8827B85F39F0B93FCCF327
:101EB000869577956795B395D9F73EF4909580957B
:101EC000709561957F4F8F4F9F4F08950E943F0DF2
:101ED00008F48FEF089516F00C94C00F0C94D60DF3
:101EE00068940C94D00D0E94000EA8F39923C1F3BE
:101EF000AEF3DF93CF931F930F93FF92C92FDD278C
:101F000088232AF02197660F771F881FDAF720E0D1
:101F100030E040E85FEB9FE3883920F0803E38F006
:101F200021968F770E94590EE8E6F0E004C00E94E7
:101F3000590EE5E9F0E00E94CE0F8B01BE01EC01E5
:101F4000FB2E6F5771097595771F880B990B0E94AF
:101F5000040D28E132E741E35FE30E94760DAF2DE7
:101F60009801AE01FF900F911F91CF91DF910E94D8
:101F7000700E0C94E70D0E943F0D880B990B08958D
:101F80009F3F31F0915020F4879577956795B795ED
:101F9000880F911D9695879597F90895DF93CF93B4
:101FA0001F930F93FF92EF92DF927B018C01689455
:101FB00006C0DA2EEF010E94760DFE01E894A5918D
:101FC0002591359145915591A6F3EF010E94700E30
:101FD000FE019701A801DA9469F7DF90EF90FF9076
:101FE0000F911F91CF91DF910895A1E21A2EAA1BA4
:101FF000BB1BFD010DC0AA1FBB1FEE1FFF1FA217B9
:10200000B307E407F50720F0A21BB30BE40BF50BB5
:10201000661F771F881F991F1A9469F7609570953E
:10202000809590959B01AC01BD01CF010895EE0F05
:10203000FF1F0590F491E02D09940F931F93CF9308
:10204000DF938230910510F482E090E0E091EE049D
:10205000F091EF0430E020E0B0E0A0E0309799F498
:102060002115310509F44AC0281B390B24303105EC
:10207000D8F58A819B816115710589F1FB019383F4
:102080008283FE0111C04081518102811381481772
:102090005907E0F04817590799F4109761F0129624
:1020A0000C93129713961C933296CF01DF91CF9128
:1020B0001F910F9108950093EE041093EF04F4CF55
:1020C0002115310551F04217530738F0A901DB0102
:1020D0009A01BD01DF01F801C1CFEF01F9CF909363
:1020E000EF048093EE04CDCFFE01E20FF31F819346
:1020F00091932250310939832883D7CF2091EC0462
:102100003091ED04232B41F4209106013091070119
:102110003093ED042093EC042091040130910501EB
:102120002115310541F42DB73EB74091080150917A
:102130000901241B350BE091EC04F091ED04E2174A
:10214000F307A0F42E1B3F0B2817390778F0AC01DA
:102150004E5F5F4F2417350748F04E0F5F1F5093B7
:10216000ED044093EC04819391939FCFF0E0E0E085
:102170009CCFCF93DF930097E9F0FC013297138255
:102180001282A091EE04B091EF04ED0130E020E066
:102190001097A1F420813181820F931F2091EC04CC
:1021A0003091ED042817390709F061C0F093ED0470
:1021B000E093EC04DF91CF910895EA01CE17DF0799
:1021C000E8F54A815B819E0141155105B1F7E901AE
:1021D000FB83EA8349915991C40FD51FEC17FD0782
:1021E00061F4808191810296840F951FE9019983A2
:1021F0008883828193819B838A83F0E0E0E012965A
:102200008D919C9113970097B9F52D913C91119761
:10221000CD010296820F931F2091EC043091ED04C2
:102220002817390739F6309751F51092EF041092BC
:10223000EE04B093ED04A093EC04BCCFD383C2832F
:1022400040815181840F951FC817D90761F44E5FF3
:102250005F4F88819981480F591F518340838A813C
:102260009B81938382832115310509F0B0CFF093D0
:10227000EF04E093EE049ECFFD01DC01C0CF13829A
:102280001282D7CFB0E0A0E0E8E4F1E10C94230E95
:102290008C01009751F4CB010E941D108C01C801E4
:1022A000CDB7DEB7E0E10C943F0EFC01E60FF71F5F
:1022B0009C0122503109E217F30708F49DC0D901AF
:1022C000CD91DC911197C617D70798F0C530D1058D
:1022D00030F3CE0104978617970708F3C61BD70B78
:1022E0002297C193D1936D937C93CF010E94B91033
:1022F000D6CF5B01AC1ABD0A4C018C0E9D1EA0917D
:10230000EE04B091EF04512C412CF12CE12C1097EC
:1023100031F58091EC049091ED048815990509F050
:102320005CC04616570608F058C080910401909191
:102330000501009741F48DB79EB740910801509177
:102340000901841B950BE817F90708F055C0F093B5
:10235000ED04E093EC04F90171836083A0CF8D91CB
:102360009C91119712966C90129713967C901397EC
:10237000A815B90559F56C0142E0C40ED11CCA1468
:10238000DB0420F1AC014A195B09DA0112961597BA
:1023900080F06282738251834083D9016D937C9374
:1023A000E114F10471F0D7011396FC93EE931297A8
:1023B00076CF22968C0F9D1FF90191838083F301C4
:1023C000EFCFF093EF04E093EE0469CF481659067F
:1023D00008F42C017D01D3019ACFCB010E941D107E
:1023E0007C01009749F0AE01B8010E94FF11C801BD
:1023F0000E94B910870153CF10E000E050CFFB01DD
:10240000DC0102C001900D9241505040D8F7089570
:10241000FB01DC018D91019080190110D9F3990B1A
:102420000895FB01DC0101900D920020E1F7089571
:1024300010E0CFE8D0E004C0FE010E941710219602
:10244000C039D107C9F7F894FFCF46000F0000004C
:10245000F0048000000000005A01BA00E700A70164
:102460001801F6000A0170756D70696E672057617A
:102470007465722E2E2E0A0050756D70696E67207D
:10248000776174657220646F6E650A00756E5072B4
:10249000657373696E672E2E2E0A00556E50726535
:1024A000737365640A00752D656E64206F66207510
:1024B0006E5072657373696E67206E6F7420646509
:1024C0007465637465640A007072657373696E671E
:1024D0002E2E2E0A00702D656E64206F662070729D
:1024E000657373696E67206E6F74206465746563CD
:1024F0007465640A0064726F7070696E672E2E2EA8
:102500000A0044726F707065640A006772696E64D5
:10251000696E672E2E2E0A004772696E64696E67B7
:1025200020446F6E650A005761726E696E672C20D9
:102530006772696E64696E6720746F6F6B20746F69
:102540006F206C6F6E67210A004F7574206F6620D4
:10255000436F666665653F0A0048656174696E672A
:1025600020746F2000726561636865642064657320
:10257000697265642074656D700A006E616E006931
:102580006E66006F766600752D546865726D6F63B8
:102590006F75706C653A20756E706C7567676564F1
:1025A000206F72206661696C65640A00702D546842
:1025B00065726D6F636F75706C653A20706F7369CB
:1025C00074696F6E696E67206F722072656C6179D5
:1025D000206661756C740A00682D74616B696E67A2
:1025E00020746F6F206C6F6E672C20636F6E746940
:1025F0006E75696E672E2E2E0A00726566696C6CA8
:1026000020636F6666656520616E642073656E6425
:1026100020636F6E7420636F6D6D616E640A00637A
:102620006F6E7400526566696C6C65640A00672D94
:102630006661696C7572653A207365636F6E6420BC
:102640006772696E64696E67206661696C75726530
:102650002C20636865636B206772696E6465722104
:102660000A00436F6D706C657465210A00417264E5
:1026700075696E6F2072756E6E696E67203A290AF1
:10268000004572726F7220686173206F63637572A8
:102690007265642E0A00436865636B206D61636830
:1026A000696E6520616E6420726573746172740A6C
:1026B00000726973740052697374726574746F0A7E
:1026C000006573707200457370726573736F0A00F2
:1026D0006C6F6E67004C756E676F0A00616D657296
:1026E00000416D65726963616E6F0A006D616B65B3
:1026F000004D616B696E6720736F6D6520636F6657
:10270000666565210A0064727972004472795275B7
:102710006E0A006E6F636F004E6F436F0A00677240
:10272000696E0070756D70007072657300756E7003
:102730007200686561740064726F7000636C65613B
:1027400000732D636C65616E0A00532D636C6561C7
:102750006E696E6720646F6E652E0A005661706F39
:0C276000722068656174696E670A0000F1
:107E0000112484B714BE81FFF0D085E080938100F7
:107E100082E08093C00088E18093C10086E0809377
:107E2000C20080E18093C4008EE0C9D0259A86E02C
:107E300020E33CEF91E0309385002093840096BBD3
:107E4000B09BFECF1D9AA8958150A9F7CC24DD24C4
:107E500088248394B5E0AB2EA1E19A2EF3E0BF2EE7
:107E6000A2D0813461F49FD0082FAFD0023811F036
:107E7000013811F484E001C083E08DD089C08234E0
:107E800011F484E103C0853419F485E0A6D080C0E4
:107E9000853579F488D0E82EFF2485D0082F10E0AE
:107EA000102F00270E291F29000F111F8ED06801E7
:107EB0006FC0863521F484E090D080E0DECF843638
:107EC00009F040C070D06FD0082F6DD080E0C81688
:107ED00080E7D80618F4F601B7BEE895C0E0D1E017
:107EE00062D089930C17E1F7F0E0CF16F0E7DF06D8
:107EF00018F0F601B7BEE89568D007B600FCFDCFD4
:107F0000A601A0E0B1E02C9130E011968C91119780
:107F100090E0982F8827822B932B1296FA010C0160
:107F200087BEE89511244E5F5F4FF1E0A038BF0790
:107F300051F7F601A7BEE89507B600FCFDCF97BE46
:107F4000E89526C08437B1F42ED02DD0F82E2BD052
:107F50003CD0F601EF2C8F010F5F1F4F84911BD097
:107F6000EA94F801C1F70894C11CD11CFA94CF0C13
:107F7000D11C0EC0853739F428D08EE10CD085E9AC
:107F80000AD08FE07ACF813511F488E018D01DD067
:107F900080E101D065CF982F8091C00085FFFCCF94
:107FA0009093C60008958091C00087FFFCCF809118
:107FB000C00084FD01C0A8958091C6000895E0E648
:107FC000F0E098E1908380830895EDDF803219F02E
:107FD00088E0F5DFFFCF84E1DECF1F93182FE3DFCA
:107FE0001150E9F7F2DF1F91089580E0E8DFEE27F6
:047FF000FF270994CA
:027FFE00040479
:00000001FF
